:0200000480007A
:100000006F00C0006F20C0276F2080279300000082
:10001000130100009301000013020000930200008E
:100020001303000093030000130400009304000076
:10003000130500009305000013060000930600005E
:100040001307000093070000130800009308000046
:100050001309000093090000130A0000930A00002E
:10006000130B0000930B0000130C0000930C000016
:10007000130D0000930D0000130E0000930E0000FE
:10008000130F0000930F000097020000938202F804
:1000900073905230177100001301412DF32240F18B
:1000A0009392C2003301510073100134EF20103AD3
:1000B00017350000130505BA6F20D01583224508B7
:1000C0007390121483204500032185008321C5000D
:1000D0000322050183224501032385018323C501F2
:1000E00003240502832445028325C5020326050354
:1000F00083264503032785038327C50303280504B7
:1001000083284504032985048329C504032A05059A
:10011000832A4505032B8505832BC505032C05067E
:10012000832C4506032D8506832DC506032E050762
:10013000832E4507032F8507832FC50703258502D7
:1001400073002010731101142322110023263100A3
:1001500023284100232A5100232C6100232E710003
:1001600023208102232291022324A1022326B1020B
:100170002328C102232AD102232CE102232EF102DB
:1001800023200105232211052324210523263105DF
:1001900023284105232A5105232C6105232E7105AF
:1001A00023208107232291072324A1072326B107B7
:1001B0002328C107232AD107232CE107232EF10787
:1001C000F312011423245100F322001023205108BC
:1001D000F322101423225108F3223014232451084F
:1001E000F322201423265108130501006F20004735
:1010000000000000000000000000000000000000E0
:1010100000000000000000000000000000000000D0
:1010200000000000000000000000000000000000C0
:1010300000000000000000000000000000000000B0
:081040000000000000000000A8
:10200000B3E7C500B367F50093F73700B306C50023
:10201000638407023386C50093070500637ED502FB
:1020200003C705009385150093871700A38FE7FE6C
:10203000E398C5FE67800000E37ED5FE93070500A8
:1020400003A70500938747009385450023AEE7FE6D
:10205000E3E8D7FE6780000067800000B367C50033
:1020600093F737003306C5006380070293F5F50F39
:10207000930705006370C50493871700A38FB7FE0D
:10208000E31CF6FE6780000093F5F50F939785003B
:10209000B3E7B70093950701B3E5F500E374C5FE18
:1020A000930705009387470023AEB7FEE3ECC7FE16
:1020B000678000006780000083470500638E07008B
:1020C0009307050003C7170093871700E31C07FE5B
:1020D0003385A7406780000013050000678000007B
:1020E00083470500938515001305150003C7F5FF09
:1020F00063880700E386E7FE3385E74067800000DA
:10210000930700006FF05FFFB367B50093F73700E8
:10211000639E07021378C6FF330805016378050341
:10212000930705006F0000019387470093854500E2
:1021300063F8070183A6070003A70500E386E6FE10
:102140003385A7403306A640138507003386C500B4
:102150006F00400103C705008347F5FF9385150015
:10216000639AE70013051500E396C5FE130500000A
:10217000678000003385E740678000009307050013
:1021800003C705009387170093851500A38FE7FE0B
:10219000E31807FE6780000003470500930600026E
:1021A000930705006318D70003C71700938717002C
:1021B000E30CD7FE9306D0026300D7069306B00265
:1021C0006300D70483C607009305000063820604FA
:1021D0001305000093871700138606FD13172500CB
:1021E00083C607003305A700131515003305A600A5
:1021F000E39206FE638005023305A040678000007D
:1022000083C617009305000093871700E39206FC2E
:10221000130500006780000083C6170093051000B7
:1022200093871700E39606FA130500006FF09FFEF0
:1022300017F6FFFF130606DD032706008327460077
:102240009355F5413367F7006306070297F6FFFFE2
:10225000938646DF9307000023A0F60013080000D2
:1022600023A2060103270600832746003367F700F1
:10227000E31207FE2320A6002322B6006F00000011
:10228000130101FF1305903423261100EFF05FFACC
:10229000130101FE1306C1001307B10113039000DF
:1022A0006F008000138707009377F500B337F300C2
:1022B000B307F04093F777029376F500938707030F
:1022C000B387F6002300F7009396C5011355450028
:1022D0009307F7FF33E5A60093D54500E314E6FC2A
:1022E0000345C100230E01006302050693050600A5
:1022F00097F6FFFF938606D117F6FFFF130686D4E5
:1023000003A7060083A74600130805009385150060
:102310003367F700B70801016302070213070000E3
:102320002320E600930700002322F60003A70600FF
:1023300083A746003367F700E31207FE03C50500D5
:1023400023A0060123A21601E31C05FA13010102D2
:102350006780000037F6FFFF3307C500B7E70300CB
:102360006370F7149356C50093820640172300004C
:10237000130343C993972200B307F30003A7070091
:102380003375C5006306070293760704638C060E57
:1023900093760708639206189306F000639ED5169D
:1023A0001367070823A0E700730005126780000089
:1023B0001747000013074704832507006384051CA3
:1023C00083A74500174600000326C6022320F70016
:1023D0006382C70C03A7050093972200B307F3009D
:1023E0001357C7001317A700136EF70D1366F701F5
:1023F00023A0C7017300051297470000938707E0E9
:1024000093963600B386D70083A706006392071E13
:1024100083A7050023A0F60083A74500B7050400A5
:1024200023A2F600F3A50510B707C0FFB307F50018
:10243000B716000013070500B386D70083AE070068
:1024400003AE470083A8870003A8C7002320D70155
:102450002322C7012324170123260701938707019D
:1024600013070701E39CD7FC739005109397220094
:10247000B307F30023A0C700730005120F1000007C
:10248000678000001367070423A0E70073000512AC
:10249000678000009747000023AE07F46FF09FF3BA
:1024A00013051004971500009385C5A897F6FFFF44
:1024B000938646B517F6FFFF1306C6B803A70600B6
:1024C00083A7460013030500938515003367F700C3
:1024D000B703010163020702930700002320F600FF
:1024E000130800002322060103A7060083A7460065
:1024F0003367F700E31207FE03C5050023A066005B
:1025000023A27600E31C05FA130101FF1305300036
:1025100023261100EFF0DFD11305100497150000FA
:10252000938585A597F6FFFF9386C6AD17F6FFFF47
:10253000130646B103A7060083A74600130E050045
:10254000938515003367F700B70E01016302070298
:10255000930700002320F600130800002322060141
:1025600003A7060083A746003367F700E31207FEC0
:1025700003C5050023A0C60123A2D601E31C05FA6A
:102580006FF09FF81305100497150000938545A37D
:1025900097F6FFFF938606A717F6FFFF130686AA96
:1025A00003A7060083A74600130F050093851500B7
:1025B0003367F700B70F01016302070293070000BA
:1025C0002320F600130800002322060103A70600BB
:1025D00083A746003367F700E31207FE03C5050033
:1025E00023A0E60123A2F601E31C05FA6FF0DFF158
:1025F00013051004971500009385059E97F6FFFFBD
:10260000938646A017F6FFFF1306C6A303A706008E
:1026100083A7460013080500938515003367F7006C
:10262000B708010163020702130700002320E60038
:10263000930700002322F60003A7060083A74600A5
:102640003367F700E31207FE03C5050023A0060168
:1026500023A21601E31C05FA6FF01FEB8325C508C2
:10266000130101FB23248104232611042322910456
:1026700023202105232E3103232C4103232A510338
:10268000232861032326710323248103232291033A
:102690002320A103232EB10193078000130405001A
:1026A0006386F516930720006380F506938745FF40
:1026B000130710006376F7009307F0006392F5228A
:1026C00003258408EFF01FC91305040003248104C7
:1026D0008320C10483244104032901048329C10305
:1026E000032A8103832A4103032B0103832BC102A5
:1026F000032C8102832C4102032D0102832DC10191
:10270000130101056FD09F9B03274508937737007E
:1027100063980708EF078000731030000327070055
:1027200083A70700630AF706130510049715000036
:102730009385059797F6FFFF9386C68C17F6FFFFE4
:102740001306469003A7060083A74600130805005A
:10275000938515003367F700B7080101630207028C
:10276000130700002320E600930700002322F60051
:1027700003A7060083A746003367F700E31207FEAE
:1027800003C5050023A0060123A21601E31C05FAD8
:1027900013053000EFF0DFA913051000EFF05FA97B
:1027A000971500009385858D1306100497F6FFFF9B
:1027B0009386468517F5FFFF1305C58803A7060016
:1027C00083A74600130E0600938515003367F700B4
:1027D000B70E010163020702930700002320F500F2
:1027E000130800002322050103A7060083A7460063
:1027F0003367F700E31207FE03C6050023A0C601F6
:1028000023A2D601E31C06FA6FF09FF8032B850282
:10281000371C0000974400009384449E171D00005D
:10282000130D4D7EB70C0400974B0000938B8BBCAF
:102830006F00C00123A2870023A08B00B717000000
:10284000330CFC00B7F703006302FC1C9357CC0069
:10285000139437003386840003260600E30006FE47
:102860009387074093972700B307FD0083A70700CE
:1028700013F60704630C06122326F100F3AD0C10C7
:10288000B707C0FFB305FC003716000013050C00A6
:102890002324B100EFF05F87630005028327C100A6
:1028A0008325810093F707086382070A3716000023
:1028B00013050C00EFF0CFF43384840073900D10F7
:1028C00083A70B0023200400E39607F69747000038
:1028D000938787B223A08B0023A087006FF01FF699
:1028E00093051004170600001306467E97E6FFFFC7
:1028F0009386467117E5FFFF1305C57403A706000D
:1029000083A7460013830500130616003367F700FC
:10291000B703010163020702930700002320F500BB
:10292000130800002322050103A7060083A7460021
:102930003367F700E31207FE8345060023A0660015
:1029400023A27600E39C05FA6FF09FE4930710043E
:10295000170600001306466F97E6FFFF9386866A08
:1029600097E5FFFF9385056E138907001306160090
:10297000B70901016F004001930700001308000030
:1029800023A0F50023A2050103A7060083A74600A4
:102990003367F700E31207FE8347060023A02601F2
:1029A00023A23601E39207FC6FF09FDE9307100429
:1029B000170600001306066697E6FFFF93868664F7
:1029C00097E5FFFF93850568138A07001306160035
:1029D000B70A01016F0040019307000013080000CF
:1029E00023A0F50023A2050103A7060083A7460044
:1029F0003367F700E31207FE8347060023A0460172
:102A000023A25601E39207FC6FF09FD813050B0039
:102A1000EFF01F82F32740F163920716172600009C
:102A20001306465E9357C600130101F69397A7005D
:102A3000232E1108232C8108971500009385855CAF
:102A400093E7170023A0F500B707002093D6C50031
:102A5000370700809387F70C232EF6FEB3E7E600D6
:102A600073900718F3260018639AD716130405000D
:102A70001347F7FF9307F00197020000938242018A
:102A8000F39252307310073B7390073A97D7BF7F8A
:102A90009387876B73905710F3270034B708C07F74
:102AA000B387170173900714B7B700009387071017
:102AB00073902730B7E701007390073073504030B0
:102AC0009737C07F93870754174700002326F79254
:102AD0009737C07F9387077217470000232CF79022
:102AE00037030800173700001307C751173E0000CF
:102AF000130ECE7093075002930500001303F303E7
:102B0000938888001396F50193D61700B366D60014
:102B100033866700B3C7F600330817011316C600E3
:102B2000939757002320C7002322070193F707023A
:102B300013078700B3E7F60093D51500E314EEFC06
:102B400013060009930500001305010097370000E4
:102B500023A4076AEFF08FD0B70700803304F40096
:102B60001305010023228108EFD04FD58320C1092E
:102B7000032481091301010A67800000B73793031A
:102B8000B70508009387E7AD130700009385C5FFDD
:102B900037080080370500406F00C0022FA00600F4
:102BA0001316F70193D61700B366D600B3C7D70044
:102BB0009397E7013376F5001357170093870600C4
:102BC0003367E600B3F6B70013F61700B3860601C5
:102BD000E31606FC03A006006FF09FFC93051004AB
:102BE000170600001306465197E6FFFF93868641BD
:102BF00017E5FFFF1305054503A7060083A7460059
:102C000013880500130616003367F700B7080101A3
:102C100063020702130700002320E500930700006A
:102C20002322F50003A7060083A746003367F700B9
:102C3000E31207FE8345060023A0060123A2160126
:102C4000E39C05FA13053000EFF08FDE678000008B
:102C500093012000930000001301100063962000F0
:102C6000631A302A63163000E39E20FE6314302A74
:102C700093013000930010001301000063962000C0
:102C8000631A302863163000E39E20FE6314302858
:102C9000930140009300F0FF1301100063962000A1
:102CA000631A302663163000E39E20FE631430263C
:102CB00093015000930010001301F0FF6396200071
:102CC000631A302463163000E39E20FE6314302420
:102CD0009301600093000000130100006394200042
:102CE0006314300063183022E39E20FE93017000CD
:102CF000930010001301100063942000631430004F
:102D0000631A3020E39E20FE930180009300F0FFC1
:102D10001301F0FF6394200063143000631C301E25
:102D2000E39E20FE93019000130200009300000038
:102D3000130100006390201E130212009302200072
:102D4000E31652FE9301A00013020000930000005E
:102D50001301000013000000639E201A13021200EA
:102D600093022000E31452FE9301B000130200000E
:102D70009300000013010000130000001300000086
:102D8000639A20181302120093022000E31252FEED
:102D90009301C00013020000930000001300000024
:102DA0001301000063982016130212009302200002
:102DB000E31452FE9301D0001302000093000000C0
:102DC000130000001301000013000000639420149E
:102DD0001302120093022000E31252FE9301E0005E
:102DE0001302000093000000130000001300000015
:102DF00013010000639020121302120093022000BE
:102E0000E31252FE9301F000130200009300000051
:102E1000130100006390201013021200930220009F
:102E2000E31652FE9301000113020000930000001C
:102E30001301000013000000639E200C1302120017
:102E400093022000E31452FE9301100113020000CC
:102E500093000000130100001300000013000000A5
:102E6000639A200A1302120093022000E31252FE1A
:102E700093012001130200009300000013000000E2
:102E8000130100006398200813021200930220002F
:102E9000E31452FE9301300113020000930000007E
:102EA00013000000130100001300000063942006CB
:102EB0001302120093022000E31252FE930140011C
:102EC0001302000093000000130000001300000034
:102ED00013010000639020041302120093022000EB
:102EE000E31252FE93001000639A000093801000DA
:102EF0009380100093801000938010009380100046
:102F000093801000930E3000930150016394D00120
:102F1000631A300013951100630005001365150056
:102F2000730000001305100073000000731000C050
:102F3000417373657274696F6E206661696C656454
:102F40003A2061646472203E3D202831554C203C7B
:102F50003C203132292026262061646472203C20E6
:102F60003633202A202831554C203C3C2031322950
:102F70000A000000417373657274696F6E206661A8
:102F8000696C65643A20212870745B315D5B616413
:102F900064722F2831554C203C3C203132295D2071
:102FA000262030783038302920262620636175733A
:102FB00065203D3D203078660A000000417373654E
:102FC0007274696F6E206661696C65643A206E6F19
:102FD00064650A00417373657274696F6E2066617F
:102FE000696C65643A20757365725F6D61707069B4
:102FF0006E675B616464722F2831554C203C3C2025
:103000003132295D2E61646472203D3D20300A001A
:10301000417373657274696F6E206661696C656473
:103020003A2070745B315D5B616464722F283155A6
:103030004C203C3C203132295D2026203078303431
:10304000300A0000417373657274696F6E206661A7
:10305000696C65643A2070745B315D5B61646472B5
:103060002F2831554C203C3C203132295D20262030
:1030700030783038300A0000417373657274696FBC
:103080006E206661696C65643A2074662D3E6570D9
:103090006320252034203D3D20300A0041737365B4
:1030A0007274696F6E206661696C65643A202122D2
:1030B000696C6C6567616C20696E7374727563749A
:1030C000696F6E220A000000417373657274696F44
:1030D0006E206661696C65643A202122756E6578A0
:1030E00070656374656420657863657074696F6E7C
:1030F000220A0000417373657274696F6E20666105
:10310000696C65643A202122756E737570706F72F8
:103110007465642073617470206D6F6465220A00A9
:040000058000000077
:00000001FF
